:020000040000FA
:02000000F42DDD
:080008008801803123309500CE
:10001000A10A063021020318A1012014A20F1328FF
:10002000A30F1328A0143D08003E031932282E1CEC
:1000300030288801880ADB308D0088018D010D157C
:10004000452301304F2300001E30A4000D1107305E
:100050004F230D1506304F23A40B26280D115328CE
:10006000452334283A2333231430A500FD01FC0135
:10007000D921DF21ED213E23210803195920013028
:10008000210203199920023021020319D9200330DB
:1000900021020319192104302102031959210530C5
:1000A0002102031999218E018C018D018E010B1102
:1000B0000900B830840015080002031C7C17B93011
:1000C000840015080002031CFC167C16BA3084005C
:1000D00015080002031CFC15BB3084001508000243
:1000E000031C7C15A330840015080002031CFD16B8
:1000F000A230840015080002031C7D16FD15A130F6
:10010000840015080002031C7D15A030840015082A
:100110000002031CFD148801880A7D088C007C08FD
:100120008D00880180308D0001308C00A50B59288E
:100130000800BC30840015080002031CFC17BD3009
:10014000840015080002031CFC16BE30840015084C
:100150000002031C7C16FC15BF3084001508000249
:10016000031C7C15A730840015080002031CFD1633
:100170007D16A630840015080002031CFD15A5306D
:10018000840015080002031C7D15A43084001508A6
:100190000002031C7D148801880A7D088C007C08FD
:1001A0008D00880140308D0002308C00A50B99280D
:1001B0000800C030840015080002031CFC17C13081
:1001C000840015080002031C7C17C2308400150847
:1001D0000002031C7C16C330840015080002031CB7
:1001E000FC157C15FD16AB30840015080002031CBD
:1001F0007D16AA30840015080002031CFD15A930E5
:10020000840015080002031CFD14A83084001508A2
:100210000002031C7D148801880A7D088C007C087C
:100220008D00880120308D0004308C00A50BD9286A
:100230000800FC17C430840015080002031C7C175A
:10024000C530840015080002031CFC16C63084006B
:1002500015080002031CFC15C730840015080002B5
:10026000031C7C15AF30840015080002031CFD162A
:10027000AE30840015080002031C7D16AD308400EA
:1002800015080002031C7D15AC308400150800021F
:10029000031CFD147D148801880A7D088C007C08ED
:1002A0008D00880110308D0008308C00A50B1929B5
:1002B0000800C830840015080002031CFC177C17D6
:1002C000C930840015080002031CFC16CA308400E3
:1002D00015080002031C7C16CB30840015080002B0
:1002E000031C7C15B330840015080002031CFD16A6
:1002F000B230840015080002031CFD15B1308400E3
:1003000015080002031C7D15FD14B030840015088B
:100310000002031C7D148801880A7D088C007C087B
:100320008D00880108308D0010308C00A50B5929F4
:100330000800CC30840015080002031CFC17CD30E7
:10034000840015080002031C7C17FC16CE308400C4
:1003500015080002031C7C16CF308400150800022B
:10036000031CFC15B730840015080002031C7D1621
:10037000B630840015080002031CFD157D15B5304C
:10038000840015080002031CFD14B4308400150815
:100390000002031C7D148801880A7D088C007C08FB
:1003A0008D00880104308D0020308C00A50B992928
:1003B00008000310260DAF00E621B200080003106C
:1003C000260D013EAF00E621B300080001308A008F
:1003D0002F08F13E03188A0A820032088A00330887
:1003E00082000234313402343C3402344434023466
:1003F0004C340234543402345C34023464340234F5
:10040000703402347434023480340234843402345C
:100410009034023494340234A0340234A4340234CC
:10042000B0340234B4340234C0340234C43402343C
:10043000D0340234D4340234E0340234E4340234AC
:10044000F0340234F4340334003403340434033419
:100450001034033414340334203403342434033488
:1004600030342D103030B1002818392A0630A6005B
:10047000322B0130A600322B2818412A0030A6006A
:10048000322B0230A600322B2818492A0030A60051
:10049000322B0330A600322B2818512A0430A60034
:1004A000322B0330A600322B2818592A0030A60020
:1004B000322B0530A600322B2818612A0730A600FF
:1004C000322B0030A600322B28186E2A003031075C
:1004D00003196C2AB10B322B2D14322BA601322BAF
:1004E0002808AC00A60A322B2C082806031D7A2AFD
:1004F000A601322B28182B10281C2B14A60A322BED
:100500002808AC00A60A322B2C082806031D8A2ACC
:10051000A601322B28182A12281C2A16A60A322BCA
:100520002808AC00A60A322B2C082806031D9A2A9C
:10053000A601322B2818AA11281CAA15A60A322BAC
:100540002808AC00A60A322B2C082806031DAA2A6C
:10055000A601322B28182A11281C2A15A60A322B8C
:100560002808AC00A60A322B2C082806031DBA2A3C
:10057000A601322B2818AA10281CAA14A60A322B6E
:100580002808AC00A60A322B2C082806031DCA2A0C
:10059000A601322B28182A10281C2A14A60A322B4E
:1005A0002808AC00A60A322B2C082806031DDA2ADC
:1005B000A601322B2818A912281CA916A60A322B2C
:1005C0002808AC00A60A322B2C082806031DEA2AAC
:1005D000A601322B28182912281C2916A60A322B0C
:1005E0002808AC00A60A322B2C082806031DFA2A7C
:1005F000A601322B2818A911281CA915A60A322BEE
:100600002808AC00A60A322B2C082806031D0A2B4A
:10061000A601322B28182911281C2915A60A322BCD
:100620002808AC00A60A322B2C082806031D1A2B1A
:10063000A601322B2818A910281CA914A60A322BAF
:100640002808AC00A60A322B2C082806031D2A2BEA
:10065000A601322B28182910281C2914A60A322B8F
:10066000A601301408002D10AD108E1E2D148E1F03
:10067000AD14080028100E1B2814080027082602B5
:10068000031C442B2608A70008002E10BD030310EE
:10069000BC0CBB0CBA0CB90C03182E140800B40027
:1006A000B40B502B0800BA01BB01BC01A030B9004B
:1006B000B709371C3A143718BA14351E3A15351ACB
:1006C000BA15B51D3A16B519BA16351D3A173519AA
:1006D000BA17B51C3B14B518BB14351C3B1535189F
:1006E000BB15B61E3B16B61ABB16361E3B17361A7E
:1006F000BB17B61D3C14B619BC14361D3C15361973
:10070000BC15B61C3C16B618BC16361C3C17361861
:10071000BC172130BD000800BE01BF010830C00079
:100720000310C20CBF0DBE0DC10CBF0DBE0DC00B22
:10073000902B0800C300C4010830C5000310C30C8F
:10074000C40DC50B9E2B44080800C6000000C60B54
:10075000A62B0800CD0A4D080F3C0319CD014D080A
:10076000B800FB01FA010800CD034D08013E031D4E
:10077000BC2B0E30CD00B800FB01FA01080029089F
:10078000CD00B800F13E031CC92B0E30CD024D0840
:10079000C22BFB01FA010800C7002010201CCE2B41
:1007A000C70BCD2B08004D0A9A23CF00D001D101F1
:1007B000D201D301D40170305718D000FF30C824C3
:1007C000CF01D001D1010130C82408000630C80093
:1007D0004330C90003104D0DFB008B1336268B17D9
:1007E000CA0003144D0DFB008B1336268B17C9006E
:1007F0004A08C800080021304802031D032C49089C
:100800007B072C24152C8B130A08CB0048087A0789
:10081000DB00031049087B07DC000318DB0A3D26D8
:10082000CC004B088A004C088B17FB0F182CFA0AD7
:100830000800230095181A2C8B13151523007B082C
:10084000910079089300230055309600AA30960055
:1008500095148B17880108008B13230095182E2CF4
:10086000151123009100230095131514230013087C
:1008700088018B17080000302C24D70008003B2487
:10088000571C442C5710452C57140030FB005708B8
:10089000F9001924D323D3230800E623FB01FA012E
:1008A000FB23CE00CE13FB23D600D60AFB23D800B1
:1008B000301C762C07302A02031D612CBF23B001A7
:1008C0004D2CAA08031D762C203029020319AA23D7
:1008D000213029020319B423003029020319CD0164
:1008E0000C30290203193F24B0014D2C2D080319A7
:1008F0008C2CD323D32303302D0203193F242D182E
:10090000842CAD18882C4D2CAA23D323D3237B2CE5
:10091000B423D323D3237B2C17304E028431031905
:10092000B52484311B304E028831031900288431EC
:100930003D08003E031DA82CA01CA82CA010571C8D
:10094000A32CAA234D2C0730B5003808B60053233A
:10095000D80B582C4D2C590D590D591A013AD91A4A
:10096000013AD919013AD9000800FB23CF00FB2333
:10097000D000FB23D100FB23D200FB23D300FB23B9
:10098000D4003030DA005608C824DA0BC32C080033
:10099000D500AE3084008001D21B8009B3308400C2
:1009A0008001521B8009AF3084008001D21A800977
:1009B000AB3084008001521A8009AA308400800183
:1009C000D2198009A2308400800152198009A33015
:1009D00084008001D2188009A73084008001521859
:1009E0008009A63084008001D31B8009A5308400D3
:1009F0008001531B8009A13084008001D31A800933
:100A0000A03084008001531A8009B2308400800134
:100A1000D3198009B7308400800153198009B6309A
:100A200084008001D3188009B130840080015318FC
:100A30008009AD3084008001D41B8009B03084006F
:100A40008001541B8009B43084008001D41A8009CD
:100A5000B53084008001541A8009AC3084008001D4
:100A6000D4198009A9308400800154198009A83064
:100A700084008001D4188009A430840080015418B7
:100A80008009CC3084008001CF1B8009C8308400ED
:100A900080014F1B8009C93084008001CF1A800972
:100AA000CA30840080014F1A8009CE308400800152
:100AB000CF198009CF30840080014F198009C130DF
:100AC00084008001CF188009BC30840080014F1859
:100AD0008009C03084008001D01B8009C4308400AC
:100AE0008001501B8009C53084008001D01A800924
:100AF000CD3084008001501A8009BB308400800111
:100B0000D0198009BA308400800150198009C3309F
:100B100084008001D0188009C630840080015018FC
:100B20008009C73084008001D11B8009CB3084004C
:100B30008001511B8009BD3084008001D11A8009D9
:100B4000B83084008001511A8009B93084008001D6
:100B5000D1198009BE308400800151198009C2304A
:100B600084008001D1188009BF30840080015118B1
:100B700080095508CC23080002302602031C03011B
:100B8000CF000030D0000130C8242D080319D82D23
:100B9000A701A6013D08003E031DC52D2D08D0006C
:100BA000CF010130C824B5010C30B6005323C52D48
:100BB000301CBC2DB001F030CF00D0017F30C824F4
:100BC000CF01D0013F30C824F030CF00D0017F30BA
:100BD000C8242908CF002A08D000FF30C824FF30DD
:100BE000C824A701A601BC2D8C019501CD01BD0132
:100BF000AB01AA01A901AC01A601A701B001A101A5
:100C0000A201A301AD0121007230990023008C01E3
:100C100022008C0122008D0123008D0121008230F1
:100C200095002100E0308E002000AD011D30D9007C
:100C30008B168B17FF30CF00D000D100FF30C824B7
:100C4000FF30C824CF01D001D101FF30C824FF30CC
:100C5000C824FF30C8243B242D08D000FF30C8240E
:100C6000FF30C8242D1C4D2C3F24BC2D48088A0081
:100C70007B08490703188A0A82000A08CB005B0830
:100C80008A005C088200093442340934D5340934BE
:100C9000EA340A347D340A3498340B342B340B3460
:100CA00040340B34A3340B34B8340B34CD340B3410
:100CB000F4340C34AB340D344A340E3437340E343F
:020CC00082347C
:101000005608D5008331FB23CF00FB23D000FB2300
:10101000D100FB23D200FB23D300FB23D400883173
:101020006430BF00AE308400D21B3A21D21F3E2173
:10103000B3308400521B3A21521F3E21AF3084004E
:10104000D21A3A21D21E3E21AB308400521A3A21E4
:10105000521E3E21AA308400D2193A21D21D3E21CF
:10106000A230840052193A21521D3E21A33084003F
:10107000D2183A21D21C3E21A730840052183A21BE
:10108000521C3E21A6308400D31B3A21D31F3E219F
:10109000A5308400531B3A21531F3E21A130840008
:1010A000D31A3A21D31E3E21A0308400531A3A218C
:1010B000531E3E21B2308400D3193A21D31D3E2164
:1010C000B730840053193A21531D3E21B6308400B5
:1010D000D3183A21D31C3E21B130840053183A2151
:1010E000531C3E21AD308400D41B3A21D41F3E2135
:1010F000B0308400541B3A21541F3E21B430840088
:10110000D41A3A21D41E3E21B5308400541A3A2113
:10111000541E3E21AC308400D4193A21D41D3E2106
:10112000A930840054193A21541D3E21A83084006E
:10113000D4183A21D41C3E21A430840054183A21FA
:10114000541C3E21CC308400CF1B3A21CF1F3E21BE
:10115000C83084004F1B3A214F1F3E21C930840004
:10116000CF1A3A21CF1E3E21CA3084004F1A3A21AD
:101170004F1E3E21CE308400CF193A21CF1D3E2193
:10118000CF3084004F193A214F1D3E21C1308400D9
:10119000CF183A21CF1C3E21BC3084004F183A2191
:1011A0004F1C3E21C0308400D01B3A21D01F3E216D
:1011B000C4308400501B3A21501F3E21C5308400AA
:1011C000D01A3A21D01E3E21CD308400501A3A2147
:1011D000501E3E21BB308400D0193A21D01D3E2143
:1011E000BA30840050193A21501D3E21C33084008A
:1011F000D0183A21D01C3E21C630840050183A2124
:10120000501C3E21C7308400D11B3A21D11F3E2102
:10121000CB308400511B3A21511F3E21BD30840048
:10122000D11A3A21D11E3E21B8308400511A3A21F8
:10123000511E3E21B9308400D1193A21D11D3E21E1
:10124000BE30840051193A21511D3E21C230840024
:10125000D1183A21D11C3E21BF30840051183A21C7
:10126000511C3E2155088331CC238831BF0B1228F5
:101270008431982C800A0319800908008008031D16
:1012800080030800173410341834803400340034DC
:1012900080340034003440340034003440340034AE
:1012A000003420340034003420340034003410344E
:1012B0000034003410340034003408340034003476
:1012C000083400340034043400340034043400346E
:1012D0000034023400340034023400340034013469
:1012E00000340034013400340034003480340034DD
:1012F000003480340034003440340034003440344E
:1013000000340034203400340034203400340034FD
:101310001034003400341034003400340834003405
:10132000003408340034003404340034003404340D
:101330000034003402340034003402340034003409
:10134000013400340034013400340034003480347B
:10135000003400348034003400344034003400342D
:10136000403400340034203400340034203400345D
:1013700000341034003400341034003400340834A5
:1013800000340034083400340034043400340034B1
:1013900004340034003402340034003402340034A5
:1013A0000034013400340034013417341034033471
:1013B000FF34FF34FF34FF34FF34FF34FF34F034A4
:1013C0000034FF34F034003400340F34FF34003480
:1013D0000F34FF341734033418348034103400349D
:1013E000803410340034403420340034403420340D
:1013F000003420344034003420344034003410347D
:101400008034003410348034003409340034003423
:101410000934003400340634003400340634003417
:1014200000348034103400348034103400344034BC
:10143000203400344034203400342034403400342C
:10144000203440340034103480340034103480347C
:1014500000340934003400340934003400340634D4
:1014600000340034063400340034003408340134CD
:1014700000340834013400340434023400340434B9
:1014800002340034023404340034023404340034AE
:10149000013408340034013408340034003490340A
:1014A00000340034903400340034603400340034AC
:1014B000603400340834013400340834013400341A
:1014C000043402340034043402340034023404346A
:1014D000003402340434003401340834003401345C
:1014E0000834003400349034003400349034003434
:1014F0000034603400340034603417341034043461
:10150000FC340F34C0340034003400340034003470
:101510000034FC340F34C0340334F0343F3400342E
:10152000003400340034003400340334F0343F34E9
:101530001B3404341834FF34FF34FF34FF34FF34D9
:10154000FF34FF34FF34FF34FF34FF34FF34FF3403
:10155000FF34FF34FF34FF34FF34FF34FF34FF34F3
:10156000FF34FF34FF3400340034003400340034DE
:1015700000340034003400340034003400340034CB
:1015800000340034003400340034003400340034BB
:10159000003400340034FF34F0340034FF34F034CD
:1015A0000034FF34F0340034FF34F0340034FF34BE
:1015B000F0340034FF34F0340034FF34F0340034BD
:1015C000FF34F0340034003400340034003400348C
:1015D000003400340034003400340034003400346B
:1015E000003400340034003400340034003400345B
:1015F00000340034003400340F34FF3400340F342E
:10160000FF3400340F34FF3400340F34FF3400341F
:101610000F34FF3400340F34FF3400340F34FF3400
:1016200000340F34FF34003400340034003400340C
:10163000003400340034003400340034003400340A
:1016400000340034003400340034003400340034FA
:10165000003400340034173403340334DB346D3485
:10166000B634DB346D34B6346D34B634DB346D34BB
:10167000B634DB34B634DB346D34B634DB346D343D
:101680001734023410348034103400348034103471
:101690000034403420340034403420340034A0344A
:1016A00050340034A034503400345034A03400346A
:1016B0005034A034003429344034003429344034C8
:1016C0000034163480340034163480340034093445
:1016D000003400340934003400340634003400345B
:1016E0000634003400340034083401340034083443
:1016F000013400340434023400340434023400343D
:101700000A34053400340A340534003405340A340C
:10171000003405340A340034023494340034023482
:1017200094340034013468340034013468340034B3
:101730000034903400340034903400340034603489
:10174000003400346034173403340334DB34603441
:101750000034DB34603400346D34B03400346D3424
:10176000B0340034B634D03400346D34B034003486
:1017700017340334033400340D34B63400340D34DC
:10178000B63400340634DB3400340634DB34003441
:101790000B346D3400340B346D3417340334063499
:1017A000C33401348634C334013486346134803424
:1017B000C33461348034C3343034C8346134303499
:1017C000C834613418346C34303418346C343034E8
:1017D0000C34363418340C3436341834863413341C
:1017E0000C34863413340C341B3404341E348034EB
:1017F00000340134003400340034C0340034033485
:10180000003400340034E034003407340034003451
:101810000034F03400340F340034003400347834B1
:1018200000341E340034003400343C3400343C3482
:101830000034003400341E34003478340034003472
:1018400000340F340034F0340034003400340734F2
:101850008134E0340034003400340334C334C03401
:101860000034003400340134E73480340034003470
:1018700000340034FF3400340034003400340034C9
:101880007E34003400340034003400343C340034FE
:101890000034003400340034183400340034003490
:1018A0000034003400340034803400340134003417
:1018B00000340034C03400340334003400340034C5
:1018C000E03400340734003400340034F0340034A1
:1018D0000F34003400340034783400341E340034C3
:1018E000003400343C3400343C34003400340034E0
:1018F0001E34003478340034003400340F340034A3
:10190000F03400340034003407348134E0340034DF
:10191000003400340334C334C034013400340034A0
:101920000134E73480340034003400340034FF34B0
:10193000003400340034003400347E340034003489
:101940000034003400343C340034003400340034BB
:101950000034183400341B3404341A348034103406
:101960000034803410340034C03430340034C03497
:1019700030340034E03470340034E03470340034F7
:10198000F034F0340034F034F03400347934E0349E
:1019900000347934E03400343F34C03400343D3412
:1019A000C03400341F34803400341F348034003499
:1019B0000F34003400340F34003400340634003463
:1019C0000034063400340034003400340034003471
:1019D0000034003400340034003400340034003467
:1019E0000034003400340034003400340034003457
:1019F000003400340034003400340834013400343E
:101A00000834013400340C34033400340C3403340F
:101A100000340E34073400340E34073400340F34ED
:101A20000F3400340F340F34003407349E34003444
:101A300007349E3400340334FC3400340334FC3463
:101A400000340134F83400340134F8340034003404
:101A5000F03400340034F0340034003460340034A6
:101A60000034603400340034003400340034003476
:101A700000340034003400340034003400340034C6
:101A800000340034003400340034003400340034B6
:101A9000003400341B34043427340634003400345A
:101AA0000634003400340F34003400340F34003472
:101AB00000341F34803400341F34803400343F3409
:101AC000C03400343D34C03400347934E034003460
:101AD0007934E0340034F034F0340034F034F0344D
:101AE0000034E03470340034E03470340034C034F6
:101AF00030340034C0343034003480341034003496
:101B000080341034003400340034003400340034A5
:101B10000034003400340034003400340034003425
:101B20000034003400340034003400340034003415
:101B300000340034003400340034603400340034A5
:101B4000603400340034F03400340034F0340034B5
:101B50000134F83400340134F83400340334FC34F4
:101B600000340334FC34003407349E34003407342A
:101B70009E3400340F340F3400340F340F340034EB
:101B80000E34073400340E34073400340C3403347C
:101B900000340C3403340034083401340034083485
:101BA0000134003400340034003400340034003494
:101BB0000034003400340034003400340034003485
:101BC0000034003400340034003400340034003475
:101BD00000340634003460340634003460340F348A
:101BE0000034F0340F340034F0341F348134F834CE
:101BF0001F348134F8343F34C334FC343F34C334AD
:101C0000FC347934E7349E347934E7349E34F0344C
:101C1000FF340F34F034FF340F34E0347E340734B3
:101C2000E0347E340734C0343C340334C0343C34B4
:101C300003348034183401348034183401340034CF
:101C400000340034003400340034003400340034F4
:101C500000340034003400340034003400340034E4
:101C600000340034003400340034003400341734BD
:101C700003340C3480341034003480341034003495
:101C800020344034003420344034003409340034EB
:101C90000034093400340034003408340134003492
:101CA000083401340034023404340034023404347F
:101CB0000034003490340034003490344034203404
:101CC0000034403420340034103480340034103474
:101CD00080340034063400340034063400340034D8
:101CE0000034043402340034043402340034013447
:101CF00008340034013408340034003460340034D3
:101D000000346034173401342134C03430340034AA
:101D1000C034303400340034003400340034003433
:101D20000034C03430340034C03430340034003433
:101D30000034003400340034003400340C340334F4
:101D400000340C34033400340034003400340034E4
:101D5000003400340C34033400340C3403340034C5
:101D600000340034003400340034003400340034D3
:101D700000340034003400340034003400340034C3
:101D80000034003400340034003400340034303483
:101D9000C03400343034C0340034003400340034F3
:101DA0000034003400343034C03400343034C034B3
:101DB0000034003400340034003400340034003483
:101DC00003340C34003403340C3400340034003455
:101DD000003400340034003403340C340034033451
:101DE0000C34003400340034003400340034003447
:101DF0000034003400340034003400340034003443
:101E00000034003400340034003400340034003432
:101E100000340F34003400340F3400340034003404
:101E2000003400340034003400340F340034003403
:101E30000F340034003400340034003400340034F3
:101E4000003400340034F03400340034F034003412
:101E50000034003400340034003400340034F034F2
:101E600000340034F03400340034003400340034E2
:101E700000340034003400340034003400340034C2
:101E800000340034003400340034003400340034B2
:061E9000003400340034B0
:020000040001F9
:02000E0084E983
:02001000FFFEF1
:02E00000FF34EB
:00000001FF
